:020000040000FA
:020000000428D2
:0800080007309F00850186010D
:1000100083168113FF308500C73086018312A50146
:100020008030A507850803191128162805182328EC
:100030008518302805193D2885196128051A742866
:10004000851A872810280130A30003302505013ABE
:1000500003194A282514A5102511A51B25154A2882
:100060000230A30003302505023A03194A2825105F
:10007000A5142511A51B25154A280430A30003301B
:100080002505033A03194A282514A5142511A51B93
:1000900025154A2808302519103086009A200508B1
:1000A00003195F28A40023082406031D58284F289D
:1000B0008601B5208508031D5A289A20102886013C
:1000C0001028250807396B20A500A5208508031DE9
:1000D00066289A201028820700340134033406343D
:1000E0000434053407340234250807397E20A5007E
:1000F000A5208508031D79289A201028820700343E
:10010000073402340134043403340634053425083A
:1001100007399120A500A5208508031D8C289A2069
:1001200010288207003402340534033404340634C2
:1001300001340734A2002F30A0001B30A100A10B16
:100140009F28A00B9D2822080800A2003F30A00095
:100150007F308616A100A10BAB288612A100A10B4F
:10016000AF28A00BA92822080800A2007F30A00019
:1001700000308616A100A10BBB28A100A10BBE2850
:100180008612A100A10BC228A100A10BC528A00BBB
:06019000B9282208080056
:041000000034003484
:02400E00103F61
:00000001FF
